:100000000C945B050C94A2050C94A2050C94A2051B
:100010000C94A2050C94A2050C94A2050C94A205C4
:100020000C94A2050C94A2050C94AB0F0C947D10BB
:100030000C94611E0C94A2050C94A2050C94A205CC
:100040000C94A2050C94A2050C94A2050C94A20594
:100050000C94A2050C94D51E0C94A2050C94A20538
:100060000C94A2050C94A2050C94A2050C94A20574
:100070000C94A2050C94A2050C94A2050C94A20564
:100080000C94A2050C94A2050C94A2050C94A20554
:100090000C94A2050C94A2050C94A2050C94A20544
:1000A0000C94A2050C94A2050C94A205EA100C1164
:1000B000FA110C11FA1151117411FA11C911DC1154
:1000C000501550157D157D15D81514160C180C18E3
:1000D0002C160C1827172717E2170C180C18F817EE
:1000E000041607090B0A1D1B06196405141A0815C6
:1000F0001C171E1F202123222E26242D25273012D7
:10010000182F0C13280F0D340E33313638111037D9
:100110002B2C352A5829787B79397A504F515272D5
:100120006C63685680668053020103555880576D92
:100130006E5462595A5B5C5D5E5F6F606174756698
:100140003E3F403C4142774476466B47804365459D
:100150008048494A4B4C3D4D3B4E3A7D7E7C7F73F7
:100160000A0025303862003A2000253032580072EB
:100170002F632030313233343536370A0061646200
:100180005F686F73745F6B62645F726563763A2059
:100190004552524F52282564290A000A002530345E
:1001A00058006164625F686F73745F6B62645F7252
:1001B0006563763A20004552524F523A206D65648D
:1001C0006961206B6579300A004552524F523A20DE
:1001D0006D65646961206B6579310A005D0A0025EF
:1001E000640020002564007C002530325800200087
:1001F00025303258006164625F6D6F7573652072DF
:1002000061773A205B000A00253031366200616474
:10021000625F686F73745F6D6F7573655F7265633E
:10022000763A2000646562756720656E61626C6570
:10023000642E0A005363616E3A20616464723A2549
:10024000642C20726567333A253034580A004166C1
:1002500074657220696E69743A0A00466F756E643F
:100260003A206D65646961206B6579730A00536398
:10027000616E3A20616464723A25642C207265676D
:10028000333A253034580A004265666F726520693A
:100290006E69743A0A005B735D004B6579626F6149
:1002A00072642073746172742E0A00555342206385
:1002B0006F6E666967757265642E0A005B575D0034
:1002C0005B535D005B525D005B445D005B435D0022
:1002D0002E0341004400420020006B0065007900BD
:1002E00062006F00610072006400200063006F0014
:1002F0006E007600650072007400650072000000F8
:100300000E0374002E006D002E006B002E00000006
:100310000403090409027400040100A03209040066
:100320000001030101000921110100012240000721
:1003300005810308000A0904010001030102000904
:100340002111010001224D000705820308000A095E
:1003500004020001030000000921110100012236FE
:10036000000705830308000A0904030002030000D4
:100370000009211101000122220007058403200049
:10038000010705040320000112011001000000080C
:10039000EDFEDB0A0101010200010631FF0974A133
:1003A000010975150026FF00952075088102097660
:1003B000150026FF00952075089102C005010980EF
:1003C000A101850216810026B7001A81002AB70014
:1003D000751095018100C0050C0901A10185031666
:1003E0000100269C021A01002A9C027510950181C9
:1003F00000C005010902A1010901A10005091901B7
:1004000029051500250195057501810295017503E2
:1004100081010501093009311581257F9502750893
:10042000810609381581257F950175088106050C1F
:100430000A38021581257F950175088106C0C0051F
:10044000010906A101050719E029E7150025019515
:1004500008750181029501750881010508190129B6
:10046000059505750191029501750391010507191F
:100470000029FF150026FF00950675088100C00AB7
:10048000002530325820006B6579626F6172645FBD
:100490007265706F72743A20004C45443A202530E2
:1004A00032580A00290A002575002F002575005DC5
:1004B0002800256400200025640020002564002019
:1004C000002564007C0025303258006D6F7573651F
:1004D0006B6579205B62746E7C7820792076206869
:1004E0005D287265702F61636C293A205B006D6B2B
:1004F0005F776865656C5F74696D655F746F5F6D6C
:100500006178203D2025640A006D6B5F7768656522
:100510006C5F6D61785F7370656564203D20256454
:100520000A006D6B5F74696D655F746F5F6D6178F4
:10053000203D2025640A006D6B5F6D61785F7370EC
:10054000656564203D2025640A006D6B5F696E74EB
:10055000657276616C203D2025640A006D6B5F64D6
:10056000656C6179203D2025640A006D6B5F7768BA
:1005700065656C5F74696D655F746F5F6D61782030
:100580003D2025640A006D6B5F776865656C5F6D63
:1005900061785F7370656564203D2025640A006D95
:1005A0006B5F74696D655F746F5F6D6178203D206E
:1005B00025640A006D6B5F6D61785F7370656564BB
:1005C000203D2025640A006D6B5F696E746572764C
:1005D000616C203D2025640A006D6B5F64656C6171
:1005E00079203D2025640A000A00257500363A204E
:1005F000776865656C5F74696D655F746F5F6D6169
:10060000783A20000A00257500353A20776865653C
:100610006C5F6D61785F73706565643A20000A00F5
:10062000257500343A2074696D655F746F5F6D6184
:10063000783A20000A00257500333A206D61785F12
:1006400073706565643A20000A00257500323A200F
:10065000696E74657276616C286D73293A20000AA0
:1006600000257500313A2064656C6179282A3130A3
:100670006D73293A20000A092D2056616C75657347
:10068000202D0A004D3E004D25643E20003F0073A2
:1006900065742064656661756C740A00433E2000D1
:1006A00077686572652064656C74613A2063757261
:1006B000736F723D25642C20776865656C3D2564F9
:1006C0000A53656520687474703A2F2F656E2E7713
:1006D000696B6970656469612E6F72672F77696BEA
:1006E000692F4D6F7573655F6B6579730A000A0931
:1006F0002D204D6F7573656B6579202D0A45534329
:100700002F713A09717569740A313A0964656C612F
:1007100079282A31306D73290A323A09696E746575
:100720007276616C286D73290A333A096D61785FBE
:1007300073706565640A343A0974696D655F746F36
:100740005F6D61780A353A09776865656C5F6D6140
:10075000785F73706565640A363A09776865656C19
:100760005F74696D655F746F5F6D61780A0A703AD6
:10077000097072696E742076616C7565730A643AEB
:10078000097365742064656661756C74730A7570AD
:100790003A092B310A646F776E3A092D310A706776
:1007A00075703A092B31300A7067646F776E3A09B9
:1007B0002D31300A0A7370656564203D2064656CD4
:1007C0007461202A206D61785F7370656564202AEA
:1007D0002028726570656174202F2074696D655FD3
:1007E000746F5F6D6178290A003F004D3E20004321
:1007F0003E20004C25640A000A092D20436F6E73C9
:100800006F6C65202D0A4553432F713A0971756944
:10081000740A6D3A096D6F7573656B65790A000A24
:10082000092D204D61676963202D0A643A096465CA
:100830006275670A783A096465627567206D61744C
:100840007269780A6B3A096465627567206B65792D
:10085000626F6172640A6D3A096465627567206D42
:100860006F7573650A763A0976657273696F6E0AF9
:10087000733A097374617475730A633A09636F6E2E
:10088000736F6C65206D6F64650A302D343A096CA6
:1008900061796572302D34284631302D4634290A6D
:1008A000506175733A09626F6F746C6F6164657241
:1008B0000A003F0074696D65725F7265616433326E
:1008C00028293A202530346C580A006B6579626F0C
:1008D0006172645F69646C653A2025580A006B6533
:1008E00079626F6172645F70726F746F636F6C3A7C
:1008F0002025580A00686F73745F6B6579626F61B9
:1009000072645F6C65647328293A2025580A000ACE
:10091000092D20537461747573202D0A00474343D9
:100920003A20342E392E32204156522D4C49424322
:100930003A20312E382E3073766E204156525F4168
:100940005243483A20617672350A004F5054494F5D
:100950004E533A204C554641204D4F5553454B453B
:10096000592045585452414B455920434F4E534FFF
:100970004C4520434F4D4D414E44204B45594D4130
:10098000505F53454354494F4E20343039360A00A6
:100990004255494C443A20383863393536312D6454
:1009A00069727479202830393A30303A343820531B
:1009B00065702032362032303136290A00564944DB
:1009C0003A2030784645454428742E6D2E6B2E29EA
:1009D000205049443A203078304144422841444232
:1009E000206B6579626F61726420636F6E766572E9
:1009F00074657229205645523A20307830313031B2
:100A00000A00444553433A20636F6E766572742042
:100A1000414442206B6579626F61726420746F207B
:100A20005553420A000A092D2056657273696F6E8C
:100A3000202D0A000A6D6F7573653A206F66660A8D
:100A4000000A6D6F7573653A206F6E0A000A6B6558
:100A500079626F6172643A206F66660A000A6B659C
:100A600079626F6172643A206F6E0A000A6D617478
:100A70007269783A206F66660A000A6D617472695D
:100A8000783A206F6E0A000A64656275673A206FD3
:100A90006E0A000A64656275673A206F66660A002E
:100AA0000A0A626F6F746C6F616465722E2E2E205D
:100AB00000433E20000011241FBECFEFDAE0DEBF6E
:100AC000CDBF04B603FE27C08091DC019091DD010B
:100AD000A091DE01B091DF018730904BA740B04B71
:100AE000D1F41092DC011092DD011092DE0110921F
:100AF000DF0114BE84B7877F84BF0FB6F894A89532
:100B000080916000886180936000109260000FBE49
:100B1000E0E0F8E3099511E0A0E0B1E0ECE7FEE4E5
:100B200002C005900D92A433B107D9F721E0A4E3E8
:100B3000B1E001C01D92AC3DB207E1F70E94DA0CB2
:100B40000C943C270C940000FF93EF93E091340148
:100B5000F0913501309709F00995EF91FF910895D3
:100B6000FC018591803011F0EFDFFBCF0895FF2766
:100B7000E0E230E247FF0CC0419597FF09C0EDE28B
:100B80006095709580959095611D711D811D911DD9
:100B900027FF02C0219530E350E2AA27660F771F96
:100BA000881F991FAA1FA41710F0A41B63955A95BC
:100BB000A9F7AA3008F0A95FA05DAF93F39561157E
:100BC00071058105910541F7ED3211F4EF93F3952D
:100BD000F21718F43F93F395FBCF8F91B5DFFA9599
:100BE000E1F70895E991F9918591803021F08532FE
:100BF00019F0AADFF9CF089520E0E8945591553215
:100C0000C1F3503311F4689455915A3348F450535A
:100C100090F3220F022E220F220F200D250FF4CF6A
:100C20000EF4219589919991533619F3533729F18F
:100C3000533559F1BC0188279927E8945C3621F493
:100C40008991999168945591543639F446EF7EF024
:100C500077FF0DC08FEF9FEF0AC055374AE039F09C
:100C6000583540E121F0523642E009F00895FF93F3
:100C7000EF937DDFEF91FF91B7CFFF93EF93FC01EF
:100C800081918030B9F360DFFBCFFF93EF9368DF92
:100C9000F1CFDF93CF93CDB7DEB72596A3DFCF910A
:100CA000DF910895282F2770E82FE695E695E695C1
:100CB000EF70F0E0E95CFE4F87FF0AC081E090E052
:100CC00001C0880F2A95EAF780959081892308C092
:100CD00081E090E001C0880F2A95EAF79081892B86
:100CE000808381E080934C0108950F931F93CF93ED
:100CF000DF93569A5E9A0E94BE092FEF87EA91E62B
:100D0000215080409040E1F700C0000088E892E068
:100D10009F938F930E9449060F900F90C1E0D0E0FF
:100D20000EE612E063E08C2F0E94C209009771F07A
:100D30009F938F93DF93CF931F930F930E94490646
:100D40000F900F900F900F900F900F909FEF29EF43
:100D500080E0915020408040E1F700C000002196E3
:100D6000C031D105F9F663E082E00E94C209813109
:100D7000910511F170F487309105F1F020F404979A
:100D80000297F0F419C089309105B1F00D97C1F4C4
:100D900013C08D31910581F030F48431910561F0FB
:100DA000499771F409C0843C910531F0873C910565
:100DB00019F0813C910521F481E080934D0102C03E
:100DC00010924D0163E087E00E94C20991E08230F9
:100DD00009F090E090934E01992341F08BE592E069
:100DE0009F938F930E9449060F900F9023E042E05B
:100DF00063E082E00E94420A8EE492E09F938F9328
:100E00000E9449060F900F90C1E0D0E004E312E089
:100E100063E08C2F0E94C209009771F09F938F931B
:100E2000DF93CF931F930F930E9449060F900F906B
:100E30000F900F900F900F908FEF99EF20E081505F
:100E400090402040E1F700C000002196C031D1055C
:100E5000F9F6E7E3F1E080E18E0F11928E13FDCFFA
:100E60008091BE0181608093BE0184E292E00E9485
:100E7000B005569A5E98DF91CF911F910F9108951A
:100E8000CF93DF938FE79BEB0197F1F700C0000052
:100E90000E943E0AEC01009711F481E0C3C097FD67
:100EA00005C080914701816080934701D7FF05C04D
:100EB000809147018E7F809347012D2F33272F7319
:100EC0003327BE016F737727C6FF02C060547109D4
:100ED000D6FF02C02054310940913601042E000C87
:100EE000550B649FC001659F900D749F900D112458
:100EF00081386FEF960714F481E89FEF9195819503
:100F0000910981386FEF960714F481E89FEF81957E
:100F100080934801249FC001259F900D349F900D20
:100F2000112481382FEF920714F481E89FEF9195F7
:100F30008195910981386FEF960714F481E89FEF4E
:100F40008195809349018091BE0183FF60C08EE04E
:100F500092E00E94B005DF93CF9388E092E09F93E8
:100F60008F930E94490686E092E00E94B00585EFCB
:100F700091E00E94B00580913601282F082E000CC8
:100F8000330B3F938F9380EF91E09F938F930E9459
:100F900049068EEE91E00E94B005809147011F92B4
:100FA0008F9389EE91E09F938F930E94490687EE7D
:100FB00091E00E94B00580914801282F082E000C76
:100FC000330B3F938F9384EE91E09F938F930E9416
:100FD000490682EE91E00E94B00580914901282FD8
:100FE000082E000C330B3F938F938FED91E09F936E
:100FF0008F930E9449068CED91E00E94B0058DB759
:101000009EB744960FB6F8949EBF0FBE8DBF87E47F
:1010100091E00E946C128091360191E088300CF0D2
:1010200090E0890F80933601DF91CF9108951F934F
:10103000CF93DF9310924C01C0910001D091010138
:101040008FEF9FEF9093010180930001CF3F8FEFCF
:10105000D80709F06AC08FE79BEB0197F1F700C052
:10106000000082E00E943B0AEC01892B09F05DC080
:1010700080914E01882309F458C087E00E943B0A02
:10108000009709F452C09C012F7733272230310595
:10109000A1F048F42115310569F02130310599F4AA
:1010A00080788A641AC02330310551F02F3731051A
:1010B000A1F009C08078826410C0807889640DC076
:1010C000807888640AC089EC91E09F938F930E9496
:1010D00049060F900F9081E18FC0292F33272F777A
:1010E00033272130310579F050F02230310579F085
:1010F0002330310581F4EC01D078D86416C0EC01BE
:10110000D078D26412C0EC01D078DA640EC0EC0161
:10111000D078D9640AC086EB91E09F938F930E94A8
:1011200049060F900F9080E167C08091BE0181FF5A
:1011300018C0209709F45DC082EA91E00E94B005D2
:10114000DF93CF938DE991E09F938F930E9449069F
:101150008BE991E00E94B0050F900F900F900F90D7
:1011600003C0209709F445C0CF379FE7D90711F492
:101170008FE705C0CF3F8FEFD80721F48FEF0E9494
:10118000520639C02D2F3327822F1C2F2F3F3105B8
:1011900081F4DF93CF938DE791E09F938F930E942B
:1011A00049060E9475060F900F900F900F908C2F9C
:1011B00023C090914D01992381F0A9014F775527C4
:1011C0004233510521F42078822F8A6006C04A30CC
:1011D000510519F42078822F82630E9452061F3F26
:1011E00051F0DC2FCC27CF6FD0930101C0930001C9
:1011F00002C080E001C081E0DF91CF911F9108958E
:10120000E82FF0E0E95CFE4F2081822F90E021E0A2
:1012100030E002C0220F331F6A95E2F728233923FA
:1012200081E0232B09F480E00895E82FF0E0E95CE9
:10123000FE4F80810895CF92DF92EF92FF920F933D
:101240001F93CF93DF938091BE0181FF35C08FE65E
:1012500091E00E94B00587E3E82E81E0F82EC0E01F
:10126000D0E09AE6C92E91E0D92E02E611E0DF9394
:10127000CF93DF92CF920E94490687E691E00E94C9
:10128000B005F70181917F010E94F61D1F928F9397
:101290001F930F930E94490680E691E00E94B005DB
:1012A00021968DB79EB708960FB6F8949EBF0FBED5
:1012B0008DBFC031D105D9F6DF91CF911F910F912C
:1012C000FF90EF90DF90CF900895682F609582E0B7
:1012D0000C947C0A509A83E091E00197F1F700C0EA
:1012E000000050989AEB9A95F1F700C00895509A33
:1012F0008AEB8A95F1F700C0509883E091E001975E
:10130000F1F700C000000895EF92FF920F931F9332
:10131000CF93DF93C0E0D0E090E8E92EF12C082FC6
:1013200010E0C7010C2E02C0959587950A94E2F74C
:1013300080239123892B19F00E94770902C00E9413
:101340006A092196C830D10561F7DF91CF911F91CD
:101350000F91FF90EF900895489B06C023E02A95D7
:10136000F1F700000197C1F70895489906C023E0FE
:101370002A95F1F700000197C1F708955898509801
:1013800008950895CF92DF92EF92FF920F931F93EB
:10139000CF93DF931F92CDB7DEB7182FF894509AF2
:1013A00083EF9BE00197F1F700C0000069830E9482
:1013B000770969816C6020E1129FC0011124862B9E
:1013C0000E9484090E946A0984EF91E00E94B50995
:1013D000892B21F4789482EE9FEF43C084EF91E053
:1013E0000E94AC09009711F478943BC011E1C12C24
:1013F000D12C02E882E890E00E94B5097C018823A4
:1014000051F199270E94AC09882329F1CC0CDD1CED
:10141000902F9E19E81A9E1518F46894C0F806C01B
:10142000113121F478948CEE9FEF1BC0115011F70D
:101430008FE591E00E94B509892B21F478948BEE19
:101440009FEF0FC08BE590E00E94AC09892BB1F7AC
:101450007894C60106C07894812F90E0919581958B
:1014600091090F90DF91CF911F910F91FF90EF9015
:10147000DF90CF90089560E00C94C20960E083E0B3
:101480000C94C2091F93CF93DF9300D01F92CDB766
:10149000DEB7182FF894509A83EF9BE00197F1F78D
:1014A00000C000002B834A8369830E947709698109
:1014B000686030E1139FC0011124862B0E948409CB
:1014C0000E946A098FE193E00197F1F700C00000E4
:1014D0000E9477094A81842F0E9484092B81822FE0
:1014E0000E9484090E946A0978940F900F900F90CF
:1014F000DF91CF911F910895262F277040E062E081
:101500000C94420A80915A0108959FB7F894109262
:1015100051019FBF9091D301943009F057C0909131
:10152000E9009F703091EC00232F217030FD20E8FE
:10153000922B24E02093E9002091EB0020FF43C090
:101540002091EE0027FF3FC020914F01222321F080
:101550002091E80025FF37C010924F0126E030911E
:10156000E80035FD15C03091D301343061F530917C
:10157000EB0035FD28C0215021F481E080934F011C
:1015800022C0EFE9FFE03197F1F700C00000E7CF9C
:101590008093F1008091E80085FD0AC08091E80009
:1015A00080FFFCCF8091E8008E778093E80006C032
:1015B0008FB7F89421E0209351018FBF9F709093D3
:1015C000E90080E008959F709093E9008FEF0895FF
:1015D000CF93DF9300D01F92CDB7DEB79C018091EF
:1015E000D301843019F593E099833B832A83909348
:1015F000E9008FEF9091E800815095FD06C095EDD0
:101600009A95F1F700008111F5CF8091E80085FFF0
:101610000DC040E050E063E070E0CE0101960E9412
:101620009B0D8091E8008E778093E8000F900F90DB
:101630000F90DF91CF910895CF93DF9300D01F9249
:10164000CDB7DEB72091D301243021F522E02983E4
:101650009B838A8383E08093E9008FEF9091E80079
:10166000815095FD06C095ED9A95F1F70000811126
:10167000F5CF8091E80085FF0DC040E050E063E0C9
:1016800070E0CE0101960E949B0D8091E8008E775C
:101690008093E8000F900F900F90DF91CF91089505
:1016A0002091D3012430F1F422E02093E9002FEFC0
:1016B0003091E800215035FD06C035ED3A95F1F73F
:1016C00000002111F5CF2091E80025FF0BC040E07C
:1016D00050E065E070E00E949B0D8091E8008E77FD
:1016E0008093E8000895CF93DF932091D3012430B5
:1016F00039F521E02093E9002FEF3091E8002150E7
:1017000035FD06C035ED3A95F1F700002111F5CF12
:101710002091E80025FF14C0EC0140E050E068E0B3
:1017200070E00E949B0D8091E8008E778093E80026
:1017300088E0FE01A2E5B1E001900D928A95E1F703
:10174000DF91CF9108958CEC92E00E94B0058091DA
:10175000D201811109C00E94300F0E948D0F80912B
:10176000E20084608093E200089588EC92E00E9499
:10177000B0051092D201089584EC92E00C94B0056B
:10178000209150012F5F822F62E30E94022799234C
:1017900019F0209350010895109250018091510149
:1017A000882371F18091D301843041F58091E90063
:1017B0008F702091EC00922F917020FD90E8892B82
:1017C00094E09093E9009091EB0090FF14C0909109
:1017D000EE0097FF10C09091E80095FF03C01092B3
:1017E000F100F9CF9091E80090FF05C09091E800DA
:1017F0009E779093E8008F708093E90010925101DA
:10180000089542E061EC81E00E94AA0E42E061ECA2
:1018100082E00E94AA0E42E061EC83E00E94AA0EE0
:1018200042E261EC84E00C94AA0E8091D5018330F1
:1018300009F453C030F4813071F0823009F48CC067
:1018400008958A3009F478C08B3009F45EC089307D
:1018500009F09AC020C08091D401813A09F094C067
:101860008091E800877F8093E8008091D801909173
:10187000D901892B21F468E082E591E003C060E0A2
:1018800080E090E070E00E94E60D8091E8008B77A8
:101890008093E80008958091D401813209F074C0EA
:1018A0008091D8019091D901892B09F06DC0809168
:1018B000E800877F8093E8008091E80082FD05C002
:1018C0008091D3018111F8CF5FC08091F1008093A6
:1018D0005A018091E8008B7753C08091D401813AFE
:1018E00009F052C08091D8019091D901892B09F05B
:1018F0004BC08091E800877F8093E8008091E800EA
:1019000080FFFCCF80910C0136C08091D4018132E0
:10191000D9F58091D8019091D901892BA9F58091B1
:10192000E800877F8093E8000E94DF0E8091D60157
:1019300080930C010C942D188091D401813221F5F3
:101940008091E800877F8093E8000E94DF0E8091FD
:10195000D70180935B0108958091D401813AA1F46D
:101960008091E800877F8093E8008091E80080FF05
:10197000FCCF80915B018093F1008091E8008E772D
:101980008093E8000C94DF0E08950895089508955B
:1019900080EC92E00E94B0050C94C70C0E94201EBF
:1019A0008091D101882329F00E944B1E81110C9453
:1019B000850D089584B7877F84BF0FB6F894A895E6
:1019C00080916000886180936000109260000FBE7B
:1019D00090E080E80FB6F8948093610090936100E6
:1019E0000FBE0E94C50C0E94A4120E94300F0E94DC
:1019F0008D0F8091E20084608093E20085E89AE098
:101A00000E94F11D78948091D3018430E1F78BEA34
:101A100092E00E94B0050E94A61282E091E00E942E
:101A200012128AE992E00E94B0050E94C60C8091D1
:101A3000D301853039F486E992E00E94B0050E9416
:101A4000CE0CF5CF0E94AC12F2CF0C945F1E8CEB43
:101A500092E00E94B0050C94250D292F33272330E6
:101A60003105C9F064F42130310581F022303105AF
:101A700009F043C084E790E024E133E042C0213222
:101A80003105F1F02232310541F137C082E190E0B9
:101A900028E833E036C099278130910541F0823043
:101AA000910541F0892B49F5E0E1F3E005C0E0E064
:101AB000F3E002C0E0EDF2E0849190E09F0121C0EC
:101AC0006430D8F4E62FF0E0EE0FFF1FEF5DFE4F1D
:101AD0002081318189E090E014C0643070F470E0BE
:101AE000FB01EE0FFF1FE75EFE4F20813181FB01FE
:101AF000EB5EFE4F808190E004C080E090E020E04B
:101B000030E0FA0131832083089580E189BD82E1CC
:101B100089BD09B400FEFDCF8091D8008F7D8093F0
:101B2000D8008091E00082608093E0008091E00026
:101B300081FDFCCF0895CF92DF92EF92FF920F9339
:101B40001F93CF93DF93EC018B016A010E94FE0E7D
:101B5000811133C0C114D10439F0F6018081918123
:101B6000081B190BC80FD91FE12CF12C0115110509
:101B700019F18091E80085FD16C08091E8008E770C
:101B80008093E800C114D10449F0F601808191816D
:101B9000E80EF91EF182E08285E00FC00E94FE0E81
:101BA000882321F30AC089918093F1000150110923
:101BB000FFEFEF1AFF0ADACF80E0DF91CF911F919C
:101BC0000F91FF90EF90DF90CF9008952091DA0170
:101BD0003091DB012617370748F06115710539F49C
:101BE0002091E8002E772093E80001C0B90140E081
:101BF00061157105A9F12091D301222309F443C095
:101C0000253009F442C02091E80023FD40C0209116
:101C1000E80022FD32C02091E80020FFE9CF40918A
:101C2000F3002091F20030E0342BFC01CF0161156C
:101C3000710559F02830310540F481918093F1000D
:101C4000615071092F5F3F4FF1CF41E028303105DE
:101C500009F040E02091E8002E772093E800C8CFFB
:101C60004111C9CF0AC08091D301882361F085302A
:101C700061F08091E80083FD0AC08091E80082FF56
:101C8000F2CF80E0089582E0089583E0089581E036
:101C900008952091DA013091DB012617370748F0CB
:101CA0006115710539F42091E8002E772093E80042
:101CB00001C0B901FC0120E06115710591F180912D
:101CC000D301882309F440C0853009F43FC08091D6
:101CD000E80083FD3DC08091E80082FD2FC0809127
:101CE000E80080FFE9CF2091F3008091F20090E0BE
:101CF000922B6115710559F08830910540F42491BB
:101D00002093F1003196615071090196F2CF21E0E4
:101D1000089709F020E08091E8008E778093E80032
:101D2000CBCF2111CCCF0AC08091D301882361F0A1
:101D3000853061F08091E80083FD0AC08091E80061
:101D400082FFF2CF80E0089582E0089583E0089555
:101D500081E00895982F973058F59093E9009817EF
:101D600039F07091EC002091ED005091F00003C02B
:101D7000242F762F50E021FF19C03091EB003E7FD9
:101D80003093EB003091ED003D7F3093ED003091CA
:101D9000EB0031603093EB007093EC002093ED008A
:101DA0005093F0002091EE0027FF07C09F5FD3CF34
:101DB0008F708093E90081E0089580E0089580911C
:101DC000D40187FF11C08091E80082FD05C0809199
:101DD000D3018111F8CF11C08091E8008B770BC03F
:101DE0008091D301882349F08091E80080FFF8CFEB
:101DF0008091E8008E778093E80008952091E400B8
:101E00003091E50095E64091EC00842F817040FF11
:101E100022C08091E80080FD1CC08091D3018823FE
:101E200091F0853091F08091EB0085FD10C04091DC
:101E3000E4005091E5004217530729F39A019150AD
:101E400011F784E0089582E0089583E0089581E029
:101E5000089580E008954091E80042FFDECF0895A4
:101E60000E949E0F0E94A60FE0EEF0E0808181604C
:101E70008083E8EDF0E080818F77808319BCA7ED47
:101E8000B0E08C918E7F8C9380818F7E80831092C6
:101E9000D20108950F931F93CF93DF930E949E0F5B
:101EA0000E94A60FC8EDD0E088818F778883888153
:101EB0008068888388818F7D888319BC1092D301C4
:101EC0001092CF011092D1011092D00100EE10E0DB
:101ED000F80180818B7F808388818160888342E0E4
:101EE00060E080E00E94AA0EE1EEF0E080818E7F4B
:101EF0008083E2EEF0E08081816080838081886071
:101F00008083F80180818E7F8083888180618883CF
:101F1000DF91CF911F910F910895E8EDF0E080815E
:101F20008F7E8083E7EDF0E080818160808384E0B4
:101F300082BF81E08093D2010C944A0FE8EDF0E07B
:101F400080818E7F80831092E20008951092DA00E3
:101F50001092E10008951F920F920FB60F92112474
:101F60002F933F934F935F936F937F938F939F93A1
:101F7000AF93BF93EF93FF938091E10082FF0BC07B
:101F80008091E20082FF07C08091E1008B7F809307
:101F9000E1000E94C00B8091DA0080FF1FC0809199
:101FA000D80080FF1BC08091DA008E7F8093DA001A
:101FB0008091D90080FF0DC080E189BD82E189BD9B
:101FC00009B400FEFDCF81E08093D3010E94A30BF2
:101FD00005C019BC1092D3010E94B50B8091E1009D
:101FE00080FF19C08091E20080FF15C08091E2005F
:101FF0008E7F8093E2008091E20080618093E20016
:102000008091D80080628093D80019BC85E08093CD
:10201000D3010E94C80C8091E10084FF30C0809100
:10202000E20084FF2CC080E189BD82E189BD09B452
:1020300000FEFDCF8091D8008F7D8093D8008091E5
:10204000E1008F7E8093E1008091E2008F7E80939B
:10205000E2008091E20081608093E2008091CF01F4
:10206000882311F084E007C08091E30087FD02C05F
:1020700081E001C083E08093D3010E94270D80910D
:10208000E10083FF29C08091E20083FF25C0809199
:10209000E100877F8093E10082E08093D30110927A
:1020A000CF018091E1008E7F8093E1008091E2007A
:1020B0008E7F8093E2008091E20080618093E20055
:1020C00042E060E080E00E94AA0E8091F00088600B
:1020D0008093F0000E94BC0BFF91EF91BF91AF91F4
:1020E0009F918F917F916F915F914F913F912F9130
:1020F0000F900FBE0F901F9018951F920F920FB662
:102100000F9211242F933F934F935F936F937F937D
:102110008F939F93AF93BF93CF93DF93EF93FF93EF
:10212000C091E900CF708091EC00D82FD17080FD74
:10213000D0E81092E9008091F000877F8093F00052
:1021400078940E94C1101092E9008091F00088609C
:102150008093F000CD2BCF70C093E900FF91EF91F9
:10216000DF91CF91BF91AF919F918F917F916F91AF
:102170005F914F913F912F910F900FBE0F901F9045
:1021800018951F93CF93DF93CDB7DEB7AA970FB6FD
:10219000F894DEBF0FBECDBFE4EDF1E088E08E0F16
:1021A0009091F10091938E13FBCF0E94150C8091BA
:1021B000E80083FF1FC18091D4019091D501492F80
:1021C00050E04A30510508F015C1FA01EA5AFF4FB4
:1021D0000C942227803881F0823809F00BC180915D
:1021E000D8018F708093E9008091EB0085FB8827F0
:1021F00080F91092E90006C08091D0019091D10140
:10220000911182609091E800977F9093E80080930D
:10221000F1001092F100C8C0282F2D7F09F0EAC00C
:10222000882319F0823061F0E5C08091D6018130B9
:1022300009F0E0C0933009F080E08093D1012BC019
:102240008091D601811127C08091D8018F7009F447
:10225000D1C08093E9002091EB0020FF1CC0933097
:1022600021F48091EB00806214C09091EB009061AA
:102270009093EB0021E030E0A90102C0440F551F0C
:102280008A95E2F74093EA001092EA008091EB0011
:1022900088608093EB001092E9008091E800877FCE
:1022A00086C08111A7C01091D6011F778091E300ED
:1022B0008078812B8093E3008091E800877F809372
:1022C000E8000E94DF0E8091E80080FFFCCF809143
:1022D000E30080688093E300111102C082E001C036
:1022E00083E08093D30186C08058823008F082C09A
:1022F0008091D6019091D7018C3D53E0950779F5F7
:1023000083E08A838AE289834FB7F894DE011396CB
:1023100020E03EE051E2E32FF0E050935700E491DB
:1023200020FF03C0E295EF703F5FEF708E2F90E0CB
:10233000EA3010F0C79601C0C0968D939D932F5F31
:10234000243149F74FBF8091E800877F8093E800F0
:102350006AE270E0CE0101960E94E60D14C0AE0163
:102360004F5F5F4F6091D8010E942D0DBC01892BFA
:1023700009F440C09091E800977F9093E80089812C
:102380009A810E94490E8091E8008B778093E80043
:1023900031C0803879F58091E800877F8093E8002C
:1023A0008091CF018093F1008091E8008E77809337
:1023B000E8000E94DF0E1EC081111CC09091D60162
:1023C0009230C0F48091E800877F8093E80090937A
:1023D000CF010E94DF0E8091CF01811106C0809154
:1023E000E30087FD02C081E001C084E08093D30157
:1023F0000E94010C8091E80083FF0AC08091E800F0
:10240000877F8093E8008091EB0080628093EB00EF
:10241000AA960FB6F894DEBF0FBECDBFDF91CF9165
:102420001F91089590936101809360010895E09158
:102430006001F0916101309721F00190F081E02D71
:10244000099480E00895EF92FF920F931F93CF932A
:10245000DF93E0916001F09161013097B1F18C015F
:102460000280F381E02D09958091BE0182FF2DC08D
:1024700080FF04C087E894E00E94B005E80118E0FE
:1024800081E8E82E84E0F82E8091BE0180FF0BC029
:1024900088811F928F93FF92EF920E9449060F90BE
:1024A0000F900F900F90115021961111EDCF809148
:1024B000BE0180FF0AC08FE794E0DF91CF911F91AA
:1024C0000F91FF90EF900C94B005DF91CF911F9189
:1024D0000F91FF90EF900895E0916001F0916101FC
:1024E000309721F00480F581E02D09940895209122
:1024F0005E0130915F018217930771F090935F0145
:1025000080935E01E0916001F0916101309721F0CC
:102510000680F781E02D0994089520915C013091A7
:102520005D018217930771F090935D0180935C01C8
:10253000E0916001F0916101309721F00084F18514
:10254000E02D0994089508950C94A3120E948A1E08
:102550000E9475060C94C109CF92DF92EF92FF9210
:102560000F931F93CF93DF9300D000D000D0CDB74F
:10257000DEB70E94170883E6C82E81E0D82E00E05F
:1025800010E0E02E802F0E941509F60141916F01A5
:10259000F42EF826B1F40F5F1F4F0031110589F7B3
:1025A0008FEF89838A831B820E94931E8160782F1C
:1025B0009D838C8349815A816B818D810E946D132B
:1025C00047C09091BE0191FF04C08E830E941B09F9
:1025D0008E8120E030E04F2D50E0922FBA01022E84
:1025E00002C0759567950A94E2F760FF2BC02983B6
:1025F000EA8221E030E0690102C0CC0CDD1C9A9532
:10260000E2F790E08C219D21892B09F420E02B83B7
:102610000E94931E8160782F9D838C8349815A810B
:102620006B818D810E946D1349815A816B817C8100
:102630008D810E940D1EF801ED59FE4F8081C82644
:10264000C08206C02F5F3F4F2830310531F6A3CF3F
:102650000E940C1E0E9454210E94400710916201AA
:102660000E941712181741F10E94171280936201FD
:102670009091BE0192FF0EC090FF0CC01F928F93ED
:1026800089E994E09F938F930E9449060F900F90E1
:102690000F900F908091620126960FB6F894DEBFDE
:1026A0000FBECDBFDF91CF911F910F91FF90EF90A3
:1026B000DF90CF900C941E1E26960FB6F894DEBFC6
:1026C0000FBECDBFDF91CF911F910F91FF90EF9083
:1026D000DF90CF9008950C946509CF93DF93CDB729
:1026E000DEB72B970FB6F894DEBF0FBECDBF942F89
:1026F0004F83252F588769877A878B874A855B8523
:10270000452B21F02F3F09F59F3FF9F4DE0111968B
:1027100086E0FD0111928A95E9F785E0FE01379682
:1027200001900D928A95E1F749815A816B817C81F4
:102730008D819E810E94C71A2B960FB6F894DEBF3A
:102740000FBECDBFDF91CF9108954F815885698528
:102750007A858B850E940D1ED9CFCF93882309F4EB
:10276000E8C0C82F8238A1F40E94171281FDE1C091
:1027700089E30E94521D0E94CB1D2FEF81EE94E051
:10278000215080409040E1F700C0000089E315C06F
:102790008338C1F40E94171280FDCBC083E50E94EC
:1027A000521D0E94CB1D2FEF81EE94E021508040FE
:1027B0009040E1F700C0000083E50E946F1DCF91BB
:1027C0000C94CB1D8438A1F40E94171282FDB1C075
:1027D00087E40E94521D0E94CB1D2FEF81EE94E0F2
:1027E000215080409040E1F700C0000087E4E5CF31
:1027F0008CEF8C0F813A48F48C2F0E947E2481113B
:1028000098C08C2F0E94521DDACF80E28C0F883046
:1028100048F4C77081E001C0880FCA95EAF70E94AA
:10282000911DCDCF8BE58C0F833078F4C53A29F01C
:10283000C63A31F083E890E005C081E890E002C03C
:1028400082E890E0CF910C94771288E58C0F853167
:1028500008F06FC0C83A61F1C93A69F1CA3A71F13A
:10286000CB3A79F1CC3A81F1CD3A89F1CE3A91F176
:10287000CF3A99F1C13BA1F1C03BA9F1C23BB1F103
:10288000C33BB9F1C43BC1F1C53BC9F1C63BD1F172
:10289000C73BD9F1C83BE1F1C93BE9F1CA3BF1F1D2
:1028A000CB3BF9F1CC3B09F43FC080E090E03EC067
:1028B00082EE90E03BC089EE90E038C08AEE90E076
:1028C00035C085EB90E032C086EB90E02FC083EB03
:1028D00090E02CC084EB90E029C087EB90E026C00C
:1028E0008CEC90E023C08DEC90E020C083E891E078
:1028F0001DC08AE891E01AC082E991E017C084E91E
:1029000091E014C081E292E011C083E292E00EC037
:1029100084E292E00BC085E292E008C086E292E099
:1029200005C087E292E002C08AE292E0CF910C9467
:102930008D12CF910895882309F466C08238A1F4DE
:102940000E94171281FF60C089E30E94521D0E94FD
:10295000CB1D2FEF81EE94E0215080409040E1F7B5
:1029600000C0000089E315C08338B9F40E94171233
:1029700080FF4AC083E50E94521D0E94CB1D2FEFAD
:1029800081EE94E0215080409040E1F700C00000CB
:1029900083E50E946F1D0C94CB1D8438A1F40E9426
:1029A000171282FF31C087E40E94521D0E94CB1D86
:1029B0002FEF81EE94E0215080409040E1F700C07D
:1029C000000087E4E6CF9CEF980F913A10F390E275
:1029D000980F983050F4877091E001C0990F8A9554
:1029E000EAF7892F0E94971DD6CF9BE5980F933069
:1029F00020F480E090E00C947712885A853120F41E
:102A000080E090E00C948D120895882321F00E94BC
:102A1000911D0C94CB1D0895882321F00E94971DD1
:102A20000C94CB1D0895CF92DF92EF92FF920F93FB
:102A30001F93CF93DF9300D000D000D0CDB7DEB787
:102A400025E0FC01DE01119601900D922A95E1F737
:102A5000FC0140813181F280258122952F706381B4
:102A60007481672B09F4D8C23F3F19F44F3F09F432
:102A7000D3C26C0149833A8389819A812E830E9453
:102A8000111D182F092F0E94101D0E94201CE02FDD
:102A9000E295EF70F0E0E05AFF4F2E810C94222770
:102AA000802F807F902F9F70092F882311F002952F
:102AB000007FFF2049F0002309F45FC2802F0E94AD
:102AC000A41D0E94CB1D59C2812F0E949B1400237C
:102AD00009F4A2C2802F0E94AA1D26960FB6F89470
:102AE000DEBF0FBECDBFDF91CF911F910F91FF9041
:102AF000EF90DF90CF900C94CB1D802F807F902F94
:102B00009F70092F803211F00295007F112319F078
:102B1000113001F129C0FF20A9F0802F222349F1B3
:102B2000213039F526960FB6F894DEBF0FBECDBF23
:102B3000DF91CF911F910F91FF90EF90DF90CF9099
:102B40000C94B41D222319F0213009F465C20E94AF
:102B5000B71D2CC0FF20E9F0263008F05DC20E94AE
:102B60008E1D802329F022C0FF20F1F0211115C015
:102B7000802F26960FB6F894DEBF0FBECDBFDF9133
:102B8000CF911F910F91FF90EF90DF90CF900C9419
:102B90000515253008F040C209C0F601858180FF87
:102BA000ECC18F708583E4CF2111FBC1802F69C1F7
:102BB000202F26952695237030E02115310521F030
:102BC00021303105C9F028C2FF2021F0812F902F3C
:102BD000937002C080E090E026960FB6F894DEBFB6
:102BE0000FBECDBFDF91CF911F910F91FF90EF905E
:102BF000DF90CF900C947712FF2021F0812F902F3F
:102C0000937002C080E090E026960FB6F894DEBF85
:102C10000FBECDBFDF91CF911F910F91FF90EF902D
:102C2000DF90CF900C948D12812FFF2019F00E941D
:102C3000DA1F02C00E94422026960FB6F894DEBF2B
:102C40000FBECDBFDF91CF911F910F91FF90EF90FD
:102C5000DF90CF900C94C720802F837009F078C04C
:102C6000F110DAC1812F829586958770880F880FC1
:102C7000912F9F70C92ED12CE12CF12C082E04C06D
:102C8000CC0CDD1CEE1CFF1C0A94D2F714FF12C002
:102C90004FE050E060E070E004C0440F551F661F35
:102CA000771F8A95D2F7CB01BA0160957095809510
:102CB000909503C060E070E0CB01202F269526950B
:102CC0002370422F50E042305105D1F0433051057E
:102CD00059F16C297D298E299F294130510541F1F7
:102CE00026960FB6F894DEBF0FBECDBFDF91CF9111
:102CF0001F910F91FF90EF90DF90CF900C94351CB7
:102D00006C297D298E299F2926960FB6F894DEBF5F
:102D10000FBECDBFDF91CF911F910F91FF90EF902C
:102D2000DF90CF900C94471C0E94351CC701B60160
:102D300026960FB6F894DEBF0FBECDBFDF91CF91C0
:102D40001F910F91FF90EF90DF90CF900C94231C78
:102D5000FF2019F0802F817001C08695882309F427
:102D60005BC1812F829586958770880F880F912F80
:102D70009F70C92ED12CE12CF12C082E04C0CC0C54
:102D8000DD1CEE1CFF1C0A94D2F714FF12C04FE0AA
:102D900050E060E070E004C0440F551F661F771FCD
:102DA0008A95D2F7CB01BA01609570958095909580
:102DB00003C060E070E0CB01202F2695269523709C
:102DC000422F50E042305105D1F04330510559F1C6
:102DD0006C297D298E299F294130510541F1269684
:102DE0000FB6F894DEBF0FBECDBFDF91CF911F911C
:102DF0000F91FF90EF90DF90CF900C94EC1C6C291A
:102E00007D298E299F2926960FB6F894DEBF0FBE26
:102E1000CDBFDF91CF911F910F91FF90EF90DF9089
:102E2000CF900C94FE1C0E94EC1CC701B6012696A4
:102E30000FB6F894DEBF0FBECDBFDF91CF911F91CB
:102E40000F91FF90EF90DF90CF900C94DA1C103F21
:102E500041F118F4103E48F48BC0123F09F450C001
:102E6000D8F1133F09F460C083C01F70802F8F71A9
:102E7000FF2021F00E94731C812F7BCE0E94941CA6
:102E8000812F26960FB6F894DEBF0FBECDBFDF911F
:102E9000CF911F910F91FF90EF90DF90CF900C9406
:102EA0000C15FF20A9F0253008F0B6C0802F8F71D7
:102EB00026960FB6F894DEBF0FBECDBFDF91CF913F
:102EC0001F910F91FF90EF90DF90CF900C94B91C61
:102ED000263008F0A1C0EACFFF20A1F0802F8F712B
:102EE00026960FB6F894DEBF0FBECDBFDF91CF910F
:102EF0001F910F91FF90EF90DF90CF900C94731C77
:102F0000FF2061F3802F8F7126960FB6F894DEBFF5
:102F10000FBECDBFDF91CF911F910F91FF90EF902A
:102F2000DF90CF900C94941CFF2091F0802F8F7134
:102F300026960FB6F894DEBF0FBECDBFDF91CF91BE
:102F40001F910F91FF90EF90DF90CF900C945E1C3B
:102F500026960FB6F894DEBF0FBECDBFDF91CF919E
:102F60001F910F91FF90EF90DF90CF900C94591C20
:102F7000FF20A1F0222309F4B1CF812F26960FB6AE
:102F8000F894DEBF0FBECDBFDF91CF911F910F919F
:102F9000FF90EF90DF90CF900C94AD13222309F4B3
:102FA000B1CF812F26960FB6F894DEBF0FBECDBFEE
:102FB000DF91CF911F910F91FF90EF90DF90CF9015
:102FC0000C949B14402F4F70612FC6010E94541F18
:102FD00026960FB6F894DEBF0FBECDBFDF91CF911E
:102FE0001F910F91FF90EF90DF90CF900C946B1B8F
:102FF000402F4F70612FC60126960FB6F894DEBFA2
:103000000FBECDBFDF91CF911F910F91FF90EF9039
:10301000DF90CF900C94571F26960FB6F894DEBF22
:103020000FBECDBFDF91CF911F910F91FF90EF9019
:10303000DF90CF9008950E94B11D0E94801D0E94D4
:10304000CB1D0E94F9210E94C72080E090E00E94E1
:10305000771280E090E00C948D120E94A11D0C94D8
:103060001B180E94111D292F22952F7030E02C3043
:1030700031054CF42A3031056CF4225031092230EC
:10308000310588F407C02C30310549F02F30310567
:1030900031F009C0803E48F0803F29F406C093FB20
:1030A000882780F9089580E0089581E00895CF93FE
:1030B000DF9300D000D01F92CDB7DEB70F900F90F6
:1030C0000F900F900F90DF91CF910895CF93DF93E2
:1030D00000D000D000D0CDB7DEB726960FB6F8945A
:1030E000DEBF0FBECDBFDF91CF9108951F93CF9369
:1030F000DF93C091730116E080917401C81799F0B5
:10310000D0E01C9FF0011D9FF00D1124EB58FE4FE5
:103110004081518162817381848195810E9466180A
:103120002196C770E9CFDF91CF911F91089540910B
:10313000A5015091A6016091A7017091A80180910D
:10314000A9019091AA010C9466188091AA01829518
:103150008F7009F054C08091A701882309F44FC0F3
:1031600080917301A09174016091A5017091A601F5
:103170004091A8015091A901B6E08A1709F43FC017
:1031800090E041155105C1F17F3F11F46F3FA1F16E
:10319000B89FF001B99FF00D1124EB58FE4F21812B
:1031A00072132AC02081621327C02281211124C0FA
:1031B000238134812417350710F421503109241B51
:1031C000350B283C3105C0F42091AA012F702061F5
:1031D0002093AA0126E0289FF001299FF00D1124D9
:1031E000E658FE4F80818F708061808385EA91E090
:1031F0000E9413150C94761801968770BECF08951F
:10320000CF92DF92EF92FF920F931F93CF93DF93B2
:10321000CDB7DEB762970FB6F894DEBF0FBECDBF55
:103220008C0185E0F801DE011D9601900D928A95D2
:10323000E1F7D8014C9111965C91119712966C911F
:1032400012971396CD90DC9014973091A501709150
:10325000A6018091A8019091A901009709F46BC182
:103260007F3F19F43F3F09F466C1E090A701EE20CB
:1032700009F4C0C02091AA01C816D90628F0F601A9
:10328000E81BF90BCF0104C0809590958C0D9D1D16
:10329000FF24F394883C910578F0F12C207F09F00D
:1032A000C6C07C2DD98AC88A89890E94571885EAA8
:1032B00091E00E941315B1C0822F807F09F046C0B3
:1032C000751314C0341312C0611110C02F70206127
:1032D0002093AA010E94971885EA91E00E94131595
:1032E0008091AA01D80115968C932EC0CD2819F192
:1032F0005F3F11F44F3FF9F0F62E61111CC0809131
:1033000073012091740136E0821709F45AC090E0ED
:10331000389FF001399FF00D1124EB58FE4F718159
:10332000571306C07081471303C07281711103C027
:1033300001968770E9CFF62E662309F418C18091B3
:10334000AA0181608093AA01F12C11C1751308C0F4
:10335000341306C0611104C08091AA01D801C3C012
:103360004D875E878D859E856A8B0E9431186A899C
:103370008823E1F16623D1F12091AA01822F829561
:103380008F7090E0029774F08091A5019091A60152
:1033900098878F831986DB86CA862C87CE0107968D
:1033A0000E94131586E0F801A5EAB1E001900D92A4
:1033B0008A95E1F70E94A5180E949718FF24F394BC
:1033C000D6C04D875E878D859E850E94111D292F51
:1033D00022952F7030E0223031050CF0BCC09F7078
:1033E00009F0B6C0805E883008F4C1C0C8010E94F0
:1033F0001315E4CFC816D90608F453C0F601E81B2C
:10340000F90BCF01883C910508F450C0F12C7C2DBC
:10341000D98AC88A89890E945718E5EAF1E086E0CE
:10342000DF011D928A95E9F70E949718A0C07513D5
:1034300014C0341312C0611110C08091AA01F801A8
:103440008583C8010E94131586E0E5EAF1E0DF01FB
:103450001D928A95E9F7FE2C8AC04D875E878D857F
:103460009E856A8B0E9431186A89882309F4BECF31
:10347000662309F4BBCF2091AA01822F82958F7019
:1034800090E002970CF48ECF8091A5019091A60157
:103490009A8389831B82DD82CC822E83CE010196A2
:1034A0007FCF809590958C0D9D1DACCFF62E662319
:1034B00009F49CCF75132EC034132CC02091AA019F
:1034C00020FD1FC0822F82958F70D9F0D8011596EC
:1034D0002C9315978F3049F08F5F982F9295907F9E
:1034E000822F8F70892B15968C93C8010E9413151B
:1034F00086E0F801A5EAB1E001900D928A95E1F726
:1035000093CF86E0F801A5EAB1E001900D928A958B
:10351000E1F72DC04D875E878D859E850E9431180D
:10352000811140CF8091AA0181608093AA01C801D6
:103530000E9413151CC0662309F458CF4D875E877F
:103540008D859E850E943118882309F44FCF2ACF9C
:10355000811148CF0CC0243031050CF047CF9F704B
:1035600009F440CFF8019581907F09F03BCF8F2D72
:1035700062960FB6F894DEBF0FBECDBFDF91CF913C
:103580001F910F91FF90EF90DF90CF9008951F93C0
:10359000CF93DF93CDB7DEB72C970FB6F894DEBF8D
:1035A0000FBECDBF4F83588769877A878B879C87EB
:1035B000CE0107960E940019882369F08F819885B3
:1035C0002A853B85232BF1F19F3F09F063C08F3F94
:1035D00009F060C037C086E0FE013796DE01119623
:1035E00001900D928A95E1F76F817885EA85FB85D8
:1035F000309741F17F3F11F46F3F21F12091740129
:1036000030E0C9010196877099274091730150E01D
:103610008417950709F447C069837A83FD83EC8397
:1036200096E0929FD001939FB00D1124AB58BE4FEE
:10363000FE01319601900D929A95E1F78093740105
:103640000E94761816E08091730190917401891799
:10365000C1F1189FC00111248B589E4F0E94001980
:10366000882379F1E09173011E9FF0011124EB583A
:10367000FE4F4081518162817381848195810E94D6
:1036800066188091730190E0019687709927809366
:103690007301D9CF4F81588569857A858B859C8543
:1036A0000E946618CFCF0E942D18109274011092BC
:1036B0007301E5EAF1E086E0DF011D928A95E9F702
:1036C000C1CF2C960FB6F894DEBF0FBECDBFDF91F1
:1036D000CF911F910895DF92EF92FF920F931F9366
:1036E000CF93DF93FC01892B09F48AC0E12CF12CE4
:1036F000DD24D394EF0121968491853709F461C0CC
:1037000058F4843708F04EC0843008F06AC0813025
:10371000D1F0823071F174C0883709F45DC050F483
:10372000863709F455C0873709F06AC08E2D0E948C
:103730009E1D54C09CE7980F903708F061C08F77AA
:103740000E949B1450C08F010E5F1F4FFE01849199
:1037500090E2980F983050F48770FD2D01C0FF0F54
:103760008A95EAF78F2F0E94A41D14C00E94AD1302
:1037700013C08F010E5F1F4FFE01C49180E28C0FBA
:10378000883060F4C7708D2D01C0880FCA95EAF7A4
:103790000E94AA1D0E94CB1DE80125C08C2F0E940B
:1037A0009B14FACF9F012E5F3F4FFE01C491CC23A3
:1037B00069F08FE99FE00197F1F700C00000C15068
:1037C000F6CF9F012E5F3F4FFE01F490E9010BC041
:1037D0000E948E1DE82E07C00E94A11D0E94CB1DD5
:1037E00002C00E94AD138F2D882341F0EFE9FFE066
:1037F0003197F1F700C000008150F6CFFE017ACF7B
:10380000DF91CF911F910F91FF90EF90DF9008957E
:103810006093AF017093B0018093B1019093B201B6
:103820000E941C1E0C941B186093AB017093AC019A
:103830008093AD019093AE010E941D1E0C941B1845
:1038400008950C94081C0F931F930091AF011091E1
:10385000B0012091B1013091B201602B712B822B0C
:10386000932B1F910F910C94081C0F931F930091A1
:10387000AF011091B0012091B1013091B2016023EC
:103880007123822393231F910F910C94081C0F9393
:103890001F930091AF011091B0012091B1013091BF
:1038A000B20160277127822793271F910F910C94F3
:1038B000081C60E070E0CB010C94141C0F931F9364
:1038C00041E050E060E070E08A019B0104C0000F1D
:1038D000111F221F331F8A95D2F7C901B8011F910A
:1038E0000F910C94141C0F931F9341E050E060E083
:1038F00070E004C0440F551F661F771F8A95D2F7EA
:103900008091AB019091AC01A091AD01B091AE015D
:103910008A019B01082B192B2A2B3B2BC901B801CB
:103920001F910F910C94141C0F931F9341E050E0D2
:1039300060E070E004C0440F551F661F771F8A9532
:10394000D2F740955095609570958091AB0190911C
:10395000AC01A091AD01B091AE018A019B01082399
:1039600019232A233B23C901B8011F910F910C94FD
:10397000141C0F931F9341E050E060E070E004C01E
:10398000440F551F661F771F8A95D2F78091AB01B0
:103990009091AC01A091AD01B091AE018A019B0163
:1039A000082719272A273B27C901B8011F910F9122
:1039B0000C94141C0F931F930091AB011091AC0158
:1039C0002091AD013091AE01602B712B822B932B96
:1039D0001F910F910C94141C0F931F930091AB0136
:1039E0001091AC012091AD013091AE0160237123A3
:1039F000822393231F910F910C94141C0F931F93F8
:103A00000091AB011091AC012091AD013091AE015C
:103A100060277127822793271F910F910C94141C04
:103A20000895CF92DF92EF92FF920F931F93CF935F
:103A3000DF938C01C090AF01D090B001E090B10154
:103A4000F090B2014091AB015091AC016091AD0199
:103A50007091AE01C42AD52AE62AF72ACFE1D0E038
:103A6000D701C6010C2E04C0B695A79597958795EA
:103A70000A94D2F780FF07C0B8018C2F0E942A1F3A
:103A80008130910531F4219758F7B80180E00E9408
:103A90002A1FDF91CF911F910F91FF90EF90DF9040
:103AA000CF90089520910D0130910E01F9013296C9
:103AB0009FEF40E05191581789F09F3F19F4511141
:103AC00001C0942F4F5F4630A9F79F3F39F0F901AD
:103AD000E90FF11D97FDFA958283089508952091CD
:103AE0000D0130910E01F9013296285F3F4F908110
:103AF000981301C010823196E217F307C1F70895B9
:103B000081E090E0E0910D01F0910E01E80FF91FC6
:103B10001082019688309105A9F708958091BD0122
:103B200008959091BD01892B8093BD0108958095E2
:103B30009091BD0189238093BD0108958093BD01BB
:103B400008951092BD0108959091BC01892B809336
:103B5000BC01089580959091BC0189238093BC019C
:103B600008951092BC0108958093B30108951092B6
:103B7000B301089580910D0190910E01FC013196E1
:103B80009C01285F3F4F80E0919191118F5FE21778
:103B9000F307D1F70895E0910D01F0910E018091A6
:103BA000BD018083E0910D01F0910E019081809123
:103BB000BC01892B80838091B301882361F0E0915F
:103BC0000D01F0910E019081892B80830E94BA1D16
:103BD00081111092B30180910D0190910E010C940E
:103BE0002312909335018093340108958295982F84
:103BF0009C7C392F36953695282F237344E0249FDB
:103C0000C0011124932F982B292F2A7A2695892FCA
:103C10008575880F822B08950895CF93DF9300D088
:103C200000D01F92CDB7DEB70F900F900F900F907E
:103C30000F90DF91CF910895089508950C946B1320
:103C40008091D301843021F11092BF0120E488E1FA
:103C500090E00FB6F894A895809360000FBE209373
:103C6000600083B7817F846083BF83B7816083BF37
:103C70007894889583B78E7F83BF0FB6F894A89504
:103C800080916000886180936000109260000FBE98
:103C9000089508950895CF930E94491E0E94170821
:103CA0000E944A1EC0E08C2F0E941509811104C099
:103CB000CF5FC031C1F701C081E0CF9108950C946E
:103CC0002D181F920F920FB60F9211248F939F936E
:103CD000AF93BF938091BF01811113C08091C00148
:103CE0009091C101A091C201B091C3014196A11D63
:103CF000B11D8093C0019093C101A093C201B09304
:103D0000C301BF91AF919F918F910F900FBE0F9004
:103D10001F90189582E084BD93E095BD9AEF97BD02
:103D200080936E0008952FB7F8948091C001909110
:103D3000C101A091C201B091C3012FBF08952FB757
:103D4000F8946091C0017091C1018091C20190917D
:103D5000C3012FBF0895CF92DF92EF92FF920F938E
:103D60001F932FB7F8944091C0015091C101609109
:103D7000C2017091C3012FBF6A017B01EE24FF24B1
:103D80008C0120E030E0C016D106E206F30610F404
:103D9000415051099A01281B390BC9011F910F91FC
:103DA000FF90EF90DF90CF9008951F920F920FB683
:103DB0000F9211248F939F93AF93BF938091C00173
:103DC0009091C101A091C201B091C3010196A11DC2
:103DD000B11D8093C0019093C101A093C201B09323
:103DE000C301BF91AF919F918F910F900FBE0F9024
:103DF0001F9018950E94300FF8942FEF87EA91E6F4
:103E0000215080409040E1F700C0000087E090EB37
:103E1000DC018093DC019093DD01A093DE01B0937F
:103E2000DF019CE088E10FB6F894A89580936000CC
:103E30000FBE90936000FFCF28E0929FF001112405
:103E4000E80FF11DE052FF4F9491892F8F709295EA
:103E50009F700895CF93C82FCB010E941C1F282F5D
:103E600030E080E1989FA0011124422B532B403871
:103E7000510519F480E090E015C09770E92FF0E04B
:103E800088E0C89FE00DF11D112484E0EE0FFF1FB4
:103E90008A95E1F7E20FF31FEE0FFF1FE050F8499C
:103EA00085919491CF91089580E090E008950895D0
:103EB0008091C60180FF0BC06091120185E0689F70
:103EC000B001112475956795759567952BC081FF95
:103ED00009C06091120185E0689FB00111247595B9
:103EE000679520C082FF07C06091120185E0689F3E
:103EF000B001112417C09091C7019923D1F06091AE
:103F00001101961788F72091120185E0289F9001F2
:103F10001124929FA001939F500D112470E0CA01BB
:103F20000E940E276038710540F46115710539F063
:103F300002C065E070E0862F08958FE7089581E064
:103F400008958091C60180FF08C06091100170E063
:103F5000759567957595679521C081FF06C060913D
:103F6000100170E07595679519C082FF04C06091DB
:103F7000100170E010C09091C7019923C1F06091C9
:103F80000F019617A0F780911001899FC00111249D
:103F900070E00E940E276038710528F461157105E4
:103FA00021F0862F08958FE7089581E0089561E05C
:103FB00070E0F4CF803F21F40E94581F819504C027
:103FC000813F29F40E94581F8093CA010895823FBF
:103FD00021F40E94581F819504C0833F29F40E9458
:103FE000581F8093C9010895893F19F40E94A11FA9
:103FF00005C08A3F31F40E94A11F81958093CB01B7
:1040000008958B3F21F40E94A11F819504C08C3F2D
:1040100029F40E94A11F8093CC010895843F21F4CC
:104020008091C801816017C0853F21F48091C8014B
:10403000826011C0863F21F48091C80184600BC06A
:10404000873F21F48091C801886005C0883F31F422
:104050008091C80180618093C80108958D3F21F44B
:104060008091C60181600BC08E3F21F48091C60112
:10407000826005C08F3F29F48091C60184608093DF
:10408000C6010895803F39F48091CA0187FF6CC052
:104090001092CA0169C0813F29F48091CA011816A3
:1040A000BCF362C09091C901823F29F497FF5CC0C4
:1040B0001092C90159C0833F19F41916CCF354C0AA
:1040C000893F41F48091CB0118160CF04DC010923D
:1040D000CB014AC08A3F29F48091CB0187FF44C0BD
:1040E000F6CF8B3F39F48091CC0187FF3DC0109211
:1040F000CC013AC08C3F29F48091CC011816BCF356
:1041000033C0843F21F48091C8018E7F17C0853F62
:1041100021F48091C8018D7F11C0863F21F48091E8
:10412000C8018B7F0BC0873F21F48091C801877F36
:1041300005C0883F31F48091C8018F7E8093C8010B
:1041400013C08D3F21F48091C6018E7F0BC08E3F3E
:1041500021F48091C6018D7F05C08F3F29F48091A5
:10416000C6018B7F8093C6018091C90181110EC069
:104170008091CA0181110AC08091CB01811106C0D2
:104180008091CC01811102C01092C70108958091E5
:10419000BE0183FF7EC08BEC94E00E94B00580914D
:1041A000C8011F928F9386EC94E09F938F930E9497
:1041B000490684EC94E00E94B0058091C901282F43
:1041C000082E000C330B3F938F9381EC94E09F9368
:1041D0008F930E9449068FEB94E00E94B005809176
:1041E000CA01282F082E000C330B3F938F938CEBC2
:1041F00094E09F938F930E9449068AEB94E00E947B
:10420000B0058091CB01282F082E000C330B3F9373
:104210008F9387EB94E09F938F930E94490685EBE1
:1042200094E00E94B0058091CC01282F082E000C4C
:10423000330B3F938F9382EB94E09F938F930E9475
:1042400049068FEA94E00E94B0058091C7011F9251
:104250008F938CEA94E09F938F930E9449068AEA99
:1042600094E00E94B0058091C6011F928F9387EA67
:1042700094E09F938F930E94490684EA94E00E9401
:10428000B0058DB79EB74C960FB6F8949EBF0FBE83
:104290008DBF88EC91E00E946C120E94931E909357
:1042A000C5018093C40108951F93CF93DF9380913C
:1042B000C4019091C5010E94AB1EAC019091C70151
:1042C000992321F02091130130E006C020911401C0
:1042D0008AE0289F900111244217530708F485C0F3
:1042E0008091C901C091CA01D091CB011091CC013C
:1042F000811107C0C11175C0D11173C0111171C0F6
:1043000074C09F3F19F09F5F9093C701181624F463
:104310000E94581F8093C9018091C90187FF05C081
:104320000E94581F81958093C9011C1624F40E9495
:10433000581F8093CA018091CA0187FF05C00E945F
:10434000581F81958093CA016091C901662331F19C
:10435000C091CA01CC2311F1062E000C770B880BFB
:10436000990B0E94092623E333E343E35FE30E94B2
:104370006D260E94D1256093C9016C2FCC0F770B5D
:10438000880B990B0E94092623E333E343E35FE3A1
:104390000E946D260E94D1256093CA011D1624F447
:1043A0000E94A11F8093CB018091CB0187FF05C0A4
:1043B0000E94A11F81958093CB01111624F40E94C5
:1043C000A11F8093CC018091CC0187FF05C00E9482
:1043D000A11F81958093CC01DF91CF911F910C9407
:1043E000C7209F3F09F08FCF97CFDF91CF911F91CB
:1043F0000895E8ECF1E085E0DF011D928A95E9F788
:104400001092C7011092C60108958EEE96E00E94A8
:10441000B0051F9281E08F931F9285E08F9380EA11
:1044200096E09F938F930E9449060F900F900F90F4
:104430000F900F900F9008958330E9F128F48130A8
:1044400061F0823009F10895853009F462C008F402
:1044500049C0863009F474C0089580911401262F54
:1044600030E0280F311D2F3F310524F4680F609391
:10447000140103C08FEF80931401809114011F92E7
:104480008F9389ED95E072C080911301262F30E063
:10449000280F311D2F3F310524F4680F609313015D
:1044A00003C08FEF80931301809113011F928F93AC
:1044B00087EC95E05BC080911201262F30E0280F39
:1044C000311D2F3F310524F4680F6093120103C0A2
:1044D0008FEF80931201809112011F928F9384EBD2
:1044E00095E044C080911101262F30E0280F311D46
:1044F0002F3F310524F4680F6093110103C08FEF43
:1045000080931101809111011F928F938FE995E0A3
:104510002DC080911001262F30E0280F311D2F3F34
:10452000310524F4680F6093100103C08FEF80936E
:104530001001809110011F928F9386E895E016C0BC
:1045400080910F01262F30E0280F311D2F3F3105BC
:1045500024F4680F60930F0103C08FEF80930F0165
:1045600080910F011F928F938BE695E09F938F931D
:104570000E9449060F900F900F900F90089583307E
:1045800081F128F4813059F08230D1F008958530DE
:1045900009F449C0B8F1863009F456C008958091F5
:1045A0001401681720F4861B8093140102C0109236
:1045B0001401809114011F928F938CE595E054C0F3
:1045C00080911301681720F4861B8093130102C0A9
:1045D00010921301809113011F928F938AE495E04A
:1045E00043C080911201681720F4861B809312014A
:1045F00002C010921201809112011F928F9387E3E3
:1046000095E032C080911101681720F4861B8093D9
:10461000110102C010921101809111011F928F931C
:1046200082E295E021C080911001681720F4861B7A
:104630008093100102C010921001809110011F920E
:104640008F9389E095E010C080910F01681720F4E6
:10465000861B80930F0102C010920F0180910F0101
:104660001F928F938EEE94E09F938F930E94490642
:104670000F900F900F900F900895CF93C82F1F9217
:104680008F9383EF97E09F938F930E94490681E079
:1046900090E0A0E0B0E0BC01CD0104C0660F771F40
:1046A000881F991FCA95D2F70E94211C0F900F9066
:1046B0000F900F90CF910C942D18CF93873288F5DF
:1046C0008E3108F00BC18E3009F487C0D8F48730E2
:1046D00009F460C08B3009F44FC0863009F002C184
:1046E0008091BE01817F8E7F8093BE0188EF97E02D
:1046F0000E94B00581EB9AE00E94B00581E08093B2
:10470000CE0146C0863109F4B0C020F4803109F4EE
:104710007AC0E8C0893109F491C08B3109F449C0ED
:10472000E1C0883349F150F4893209F4D5C08533AA
:1047300009F4D2C0873209F0D5C0CEC0833409F461
:10474000CBC028F48A3308F4CDC08953C8C088345C
:1047500009F0C8C00E942D1880EA9AE00E94B005B6
:104760002FEF83ED90E3215080409040E1F700C0AF
:1047700000000E94FA1E0CC08FE198E041C087E85B
:104780009AE00E94B0058091BE0181608093BE01D5
:10479000C1E0ADC08091BE01C82FC17080FFEFCFD6
:1047A00083E99AE00E94B0058091BE01817F8E7FEF
:1047B0003FC09091BE0191FBCC27C0F981E0C82792
:1047C000892FC0FB81F98093BE01CC2319F08AE7C1
:1047D0009AE029C08CE69AE013C09091BE0192FB4A
:1047E000CC27C0F981E0C827892FC0FB82F98093CC
:1047F000BE01CC2319F08DE59AE015C08DE49AE056
:104800000E94B005C5CF9091BE0193FBCC27C0F9A3
:1048100081E0C827892FC0FB83F98093BE01CC2398
:1048200051F081E49AE00E94B0058091BE01816060
:104830008093BE015CC084E39AE0E2CF85E29AE017
:104840000E94B00582E09AE00E94B0058DEB99E0ED
:104850000E94B00580E999E00E94B0058BE499E0E0
:104860000E94B0058DE199E0CBCF8FE099E00E94E6
:10487000B0050E9417121F928F9385EF98E09F93C7
:104880008F930E94490680910C011F928F938EEDA9
:1048900098E09F938F930E94490680915B011F923D
:1048A0008F938BEC98E09F938F930E9449060E9410
:1048B0009F1E9F938F937F936F9384EB98E09F93BA
:1048C0008F930E9449068DB79EB742960FB6F89413
:1048D0009EBF0FBE8DBF5CCF80E001C08D510E9496
:1048E0003D2356CF82EB98E00E94B005C0E08C2FAC
:1048F000CF91089580E0089580E00895CF93C82F68
:104900008091CE01813069F020F0823009F449C0F5
:1049100040C167E08FE00E940009882309F43FC18D
:1049200006C067E08FE00E940009882361F08C2FA9
:104930000E947A24811104C08C2F0E945D232FC015
:1049400081E090E02CC08C2F0E947C24811126C035
:10495000C431E1F070F4CB3081F0C031D1F40E9469
:1049600005228BEE97E00E94B00582E08093CE0195
:1049700015C0C93259F0C83361F488EF97E00E943E
:10498000B0058FEE97E00E94B00508C01092CE01EE
:1049900004C189EE97E00E94B005FFC081E08170FC
:1049A000FEC0C43228F5CE3108F0C1C0CB30A1F131
:1049B000D0F4C73009F0D3C08EE18093140182E3B4
:1049C000809313018AE08093120184E180931101A6
:1049D00088E08093100188E280930F018FE896E0D1
:1049E0000E94B005BFC0C33149F1C431C1F0B7C0A6
:1049F000CB3409F4A9C028F4C93289F0C83361F076
:104A0000AEC0C13509F49EC0C23509F499C0CE3498
:104A100009F0A5C06AE09EC00E940522A3C0809153
:104A2000CD01882319F01092CD019CC08CE996E04D
:104A30000E94B00581E08093CE01B1C086E796E088
:104A40000E94B00584E696E00E94B00580911401B2
:104A50001F928F9381E696E09F938F930E94490661
:104A60008FE596E00E94B0058DE496E00E94B005C7
:104A7000809113011F928F938AE496E09F938F9306
:104A80000E94490688E496E00E94B00589E396E01A
:104A90000E94B005809112011F928F9386E396E0E9
:104AA0009F938F930E94490684E396E00E94B0058D
:104AB00083E296E00E94B005809111011F928F93CE
:104AC00080E296E09F938F930E9449068EE196E0E4
:104AD0000E94B00589E096E00E94B0058091100127
:104AE0001F928F9386E096E09F938F930E944906D2
:104AF00084E096E00E94B0058DEE95E00E94B0053E
:104B000080910F011F928F938AEE95E09F938F9370
:104B10000E94490688EE95E00E94B0058DB79EB7C9
:104B200048960FB6F8949EBF0FBE8DBF1BC0CE51E6
:104B3000EC2FF0E0E75DFE4F80818093CD0112C045
:104B400061E003C061E006C06AE08091CD010E948F
:104B50001C2208C08091CD010E94BF2203C08DE8B5
:104B600096E013C08091CD01882369F01F928F9346
:104B700087E896E09F938F930E9449060F900F90CD
:104B80000F900F9004C084E896E00E94B00581E089
:104B900006C01092CE0180E002C080E000CFCF912D
:104BA00008950E94D8256894B1110C946726089541
:104BB0000E944C2688F09F5798F0B92F9927B7513B
:104BC000B0F0E1F0660F771F881F991F1AF0BA95B1
:104BD000C9F714C0B13091F00E946626B1E0089583
:104BE0000C946626672F782F8827B85F39F0B93F75
:104BF000CCF3869577956795B395D9F73EF4909564
:104C00008095709561957F4F8F4F9F4F0895E894E1
:104C100009C097FB3EF490958095709561957F4F04
:104C20008F4F9F4F9923A9F0F92F96E9BB279395B2
:104C3000F695879577956795B795F111F8CFFAF4C2
:104C4000BB0F11F460FF1BC06F5F7F4F8F4F9F4FF3
:104C500016C0882311F096E911C0772321F09EE851
:104C6000872F762F05C0662371F096E8862F70E0B7
:104C700060E02AF09A95660F771F881FDAF7880F91
:104C80009695879597F9089557FD9058440F551FAD
:104C900059F05F3F71F04795880F97FB991F61F0BE
:104CA0009F3F79F087950895121613061406551F35
:104CB000F2CF4695F1DF08C0161617061806991FA1
:104CC000F1CF86957105610508940895E894BB2796
:104CD00066277727CB0197F908950E9480260C94C8
:104CE000F1260E94E32638F00E94EA2620F0952360
:104CF00011F00C94DA260C94E02611240C9467260B
:104D00000E94442670F3959FC1F3950F50E0551F04
:104D1000629FF001729FBB27F00DB11D639FAA2710
:104D2000F00DB11DAA1F649F6627B00DA11D661F5F
:104D3000829F2227B00DA11D621F739FB00DA11D80
:104D4000621F839FA00D611D221F749F3327A00D3A
:104D5000611D231F849F600D211D822F762F6A2FD6
:104D600011249F5750409AF0F1F088234AF0EE0F3B
:104D7000FF1FBB1F661F771F881F91505040A9F768
:104D80009E3F510580F00C94DA260C9467265F3F15
:104D9000E4F3983ED4F3869577956795B795F795A4
:104DA000E7959F5FC1F7FE2B880F911D969587951C
:104DB00097F9089597F99F6780E870E060E008959B
:104DC0009FEF80EC089500240A9416161706180623
:104DD0000906089500240A941216130614060506FF
:104DE0000895092E0394000C11F4882352F0BB0F90
:104DF00040F4BF2B11F460FF04C06F5F7F4F8F4FF3
:104E00009F4F0895991B79E004C0991F961708F0E9
:104E1000961B881F7A95C9F78095089597FB072EF2
:104E200016F4009407D077FD09D00E94282707FCCC
:104E300005D03EF4909581959F4F089570956195AA
:104E40007F4F0895EE0FFF1F0590F491E02D099418
:104E5000AA1BBB1B51E107C0AA1FBB1FA617B707A0
:104E600010F0A61BB70B881F991F5A95A9F78095BC
:0C4E70009095BC01CD010895F894FFCF8F
:104E7C00FFFF820A730B500B1C0BE80A01B40128CC
:104E8C0008140A321E404D36223F04F203BC039A2A
:104E9C000326033F035803710301020304050607AD
:044EAC0008090000F1
:106800000000EA44E944E2440400050006000700F1
:10681000080009000A000B000C000D000E000F001C
:1068200010001100120013001400150016001700CC
:10683000180019001A001B001C001D001E001F007C
:10684000200021002200230024002500260027002C
:10685000280029002A002B002C002D002E002F00DC
:10686000300031A132003300340035A1360037004A
:10687000380082003A003B003C003D003E003F00F3
:1068800040004100420043004400450046004700EC
:10689000480049004A004B004C004D004E004F009C
:1068A000500051005200530067005400550056003C
:1068B000580059005A005B005C005D005E005F00FC
:1068C0006000610062006300640000005700000087
:1068D000CD440000000000000000000000000000A7
:1068E0000000000000007300000000000000000035
:1068F000E000E100E200E300E400E500E600E7007C
:106900000100010001000100EA4401000100E2442D
:106910000100010001000100460001004A004B0097
:10692000010001004700480001000100E9440100A6
:106930000100010001000100010001003A003B00DC
:106940003C003D003E003F0040004100420043004B
:10695000010001004C00010001004400450052000C
:1069600049000100010050004F0001004D004E00A1
:1069700051000100010001000100010001000100BF
:1069800001000100010001000100010001000100FF
:1069900001000100010001000100010001004D00A3
:1069A0004A004E004B0001000100010001000100FF
:1069B00001000100010001000100010001000100CF
:1069C00001000100010001000100010001000100BF
:1069D00001000100010001000100010001000100AF
:1069E000010001000100010001000100010001009F
:1069F000010001000100010001000100010001008F
:00000001FF
